 SWDialParserG

 Timestamp is 54004926 (Fri Aug 29 17:34:30 2014)

 Preferred load address is 00100000

 Start         Length     Name                   Class
 0001:00000000 00005794H .text                   CODE
 0001:00005794 00000090H .text$yc                CODE
 0001:00005824 00000058H .text$yd                CODE
 0002:00000000 00001424H .rdata                  DATA
 0002:00001424 0000016cH .rdata$r                DATA
 0002:00001590 00000090H .xdata                  DATA
 0002:00001620 000000e8H .xdata$x                DATA
 0002:00001708 00000000H ATL$__a                 DATA
 0002:00001708 00000000H ATL$__z                 DATA
 0002:00001708 00000078H .idata$2                DATA
 0002:00001780 00000014H .idata$3                DATA
 0002:00001794 00000138H .idata$4                DATA
 0002:000018cc 00000120H .idata$6                DATA
 0002:000019f0 0000014cH .edata                  DATA
 0003:00000000 00000138H .idata$5                DATA
 0003:00000138 00000004H .CRT$XCA                DATA
 0003:0000013c 00000004H .CRT$XCAA               DATA
 0003:00000140 00000004H .CRT$XCL                DATA
 0003:00000144 00000008H .CRT$XCU                DATA
 0003:0000014c 00000004H .CRT$XCZ                DATA
 0003:00000150 00000004H .CRT$XIA                DATA
 0003:00000154 00000004H .CRT$XIZ                DATA
 0003:00000158 00000004H .CRT$XPA                DATA
 0003:0000015c 00000004H .CRT$XPZ                DATA
 0003:00000160 00000004H .CRT$XTA                DATA
 0003:00000164 00000004H .CRT$XTZ                DATA
 0003:00000168 000000bcH .data                   DATA
 0003:00000228 000004c9H .bss                    DATA
 0004:00000000 00000508H .pdata                  DATA
 0005:00000000 000000a0H .rsrc$01                DATA
 0005:000000a0 00000500H .rsrc$02                DATA

  Address         Publics by Value              Rva+Base       Lib:Object

 0000:00000000       ___safe_se_handler_count   00000000     <absolute>
 0000:00000000       ___safe_se_handler_table   00000000     <absolute>
 0001:00000000       ?AddRef@CSWContextMenuClassFactory@@UAAKXZ 00101000 f   clsfact.obj
 0001:0000001c       ?CreateInstance@CSWContextMenuClassFactory@@UAAJPAUIUnknown@@ABU_GUID@@PAPAX@Z 0010101c f   clsfact.obj
 0001:000000a8       ?LockServer@CSWContextMenuClassFactory@@UAAJH@Z 001010a8 f   clsfact.obj
 0001:000000b0       ?Release@CSWContextMenuClassFactory@@UAAKXZ 001010b0 f   clsfact.obj
 0001:000000fc       ?QueryInterface@CSWContextMenuClassFactory@@UAAJABU_GUID@@PAPAX@Z 001010fc f   clsfact.obj
 0001:000001a0       ??0CSWContextMenuClassFactory@@QAA@XZ 001011a0 f   clsfact.obj
 0001:000001cc       ?SWDialParserWndProc@@YAJPAUHWND__@@IIJ@Z 001011cc f   DialParsExtOEM.obj
 0001:00000364       ?LaunchRiltest@@YAXXZ      00101364 f   DialParsExtOEM.obj
 0001:000003e8       ?LaunchRegEdit@@YAXXZ      001013e8 f   DialParsExtOEM.obj
 0001:0000046c       ?LaunchPhoneUtility@@YAKPBG@Z 0010146c f   DialParsExtOEM.obj
 0001:000004fc       ?CreateMessageWindow@@YAJPAPAUHWND__@@PAUHINSTANCE__@@@Z 001014fc f   DialParsExtOEM.obj
 0001:00000638       DllMain                    00101638 f   DialParsExtOEM.obj
 0001:000006e8       ?SW_PhExtFormatPhoneNumber@@YAHPBG00K@Z 001016e8 f   DialParsExtOEM.obj
 0001:000006f8       ?CheckifEmergencyNumber@@YAHPAG@Z 001016f8 f   DialParsExtOEM.obj
 0001:00000880       ?CheckIfSpecialNumber@@YAHPAG@Z 00101880 f   DialParsExtOEM.obj
 0001:000008e0       ?CheckforRoamGuard@@YAHPAUHWND__@@@Z 001018e0 f   DialParsExtOEM.obj
 0001:000009e4       ?MakeTapiVoiceCall@@YAKPAGI@Z 001019e4 f   DialParsExtOEM.obj
 0001:00000a6c       ?CheckPowerState@@YAXXZ    00101a6c f   DialParsExtOEM.obj
 0001:00000aa8       DllCanUnloadNow            00101aa8 f   DialParsExtOEM.obj
 0001:00000ac4       DllGetClassObject          00101ac4 f   DialParsExtOEM.obj
 0001:00000b3c       ?AddRef@Csw_ctxMenu@@UAAKXZ 00101b3c f   DialParsExtOEM.obj
 0001:00000b50       ?QueryInterface@Csw_ctxMenu@@UAAJABU_GUID@@PAPAX@Z 00101b50 f   DialParsExtOEM.obj
 0001:00000c20       ?InvokeCommand@Csw_ctxMenu@@UAAJPAU_CMInvokeCommandInfo@@@Z 00101c20 f   DialParsExtOEM.obj
 0001:00000c6c       ?QueryContextMenu@Csw_ctxMenu@@UAAJPAUHMENU__@@IIII@Z 00101c6c f   DialParsExtOEM.obj
 0001:00000cd8       ?GetSite@Csw_ctxMenu@@UAAJABU_GUID@@PAPAX@Z 00101cd8 f   DialParsExtOEM.obj
 0001:00000d18       ?SetSite@Csw_ctxMenu@@UAAJPAUIUnknown@@@Z 00101d18 f   DialParsExtOEM.obj
 0001:00000d58       ?LaunchActWiz@@YAXXZ       00101d58 f   DialParsExtOEM.obj
 0001:00000df8       ?AddRef@Csw_ctxMenu@@W3AAKXZ 00101df8 f i DialParsExtOEM.obj
 0001:00000e00       ?QueryInterface@Csw_ctxMenu@@W3AAJABU_GUID@@PAPAX@Z 00101e00 f i DialParsExtOEM.obj
 0001:00000e08       ?PhExtFormatPhoneNumber@@YAHPBG00K@Z 00101e08 f   DialParsExtOEM.obj
 0001:00000e18       ?SW_IsImmediateDialRequestRequired@@YAHPBG@Z 00101e18 f   DialParsExtOEM.obj
 0001:00000f44       ?CheckSpecialProcess@@YAHPAG@Z 00101f44 f   DialParsExtOEM.obj
 0001:0000100c       ?Release@Csw_ctxMenu@@UAAKXZ 0010200c f   DialParsExtOEM.obj
 0001:00001060       ?GetCommandString@Csw_ctxMenu@@UAAJIIPAIPADI@Z 00102060 f   DialParsExtOEM.obj
 0001:00001104       ?Release@Csw_ctxMenu@@W3AAKXZ 00102104 f i DialParsExtOEM.obj
 0001:0000110c       ?IsImmediateDialRequestRequired@@YAHPBG@Z 0010210c f   DialParsExtOEM.obj
 0001:00001198       ?SW_PreprocessDialRequest@@YAKPAUHWND__@@PBGH@Z 00102198 f   DialParsExtOEM.obj
 0001:0000142c       ??0Csw_ctxMenu@@QAA@XZ     0010242c f   DialParsExtOEM.obj
 0001:000014e8       ?PreprocessDialRequest@@YAKPAUHWND__@@PBGH@Z 001024e8 f   DialParsExtOEM.obj
 0001:000014f4       ?Init@CComCriticalSection@ATL@@QAAJXZ 001024f4 f i resultelement.obj
 0001:0000154c       ??0CResultListElement@@QAA@XZ 0010254c f   resultelement.obj
 0001:00001564       ??1CResultListElement@@UAA@XZ 00102564 f   resultelement.obj
 0001:00001574       ?SetCallBackId@CResultListElement@@QAAXJ@Z 00102574 f   resultelement.obj
 0001:0000157c       ?GetCallBackId@CResultListElement@@QAAJXZ 0010257c f   resultelement.obj
 0001:00001584       ?SetFuncId@CResultListElement@@QAAXW4eFuncId@1@@Z 00102584 f   resultelement.obj
 0001:0000158c       ?GetFuncId@CResultListElement@@QAA?AW4eFuncId@1@XZ 0010258c f   resultelement.obj
 0001:00001594       ??_GCResultListElement@@UAAPAXI@Z 00102594 f i resultelement.obj
 0001:00001594       ??_ECResultListElement@@UAAPAXI@Z 00102594 f i resultelement.obj
 0001:000015b8       ??1bad_alloc@std@@UAA@XZ   001025b8 f i winmodemstat.obj
 0001:000015cc       ??_Gbad_alloc@std@@UAAPAXI@Z 001025cc f i winmodemstat.obj
 0001:000015cc       ??_Ebad_alloc@std@@UAAPAXI@Z 001025cc f i winmodemstat.obj
 0001:000015fc       ??0CModemStatus@@QAA@XZ    001025fc f   winmodemstat.obj
 0001:00001654       ?Deregister@CModemStatus@@SAXXZ 00102654 f   winmodemstat.obj
 0001:00001680       ?Send2UI@CModemStatus@@SAJIIJ@Z 00102680 f   winmodemstat.obj
 0001:00001748       ?UpdateCallTypeAndStatus@CModemStatus@@KAKKKG@Z 00102748 f   winmodemstat.obj
 0001:00001c40       ??8?$_Const_iterator@$00@?$list@VCResultListElement@@V?$allocator@VCResultListElement@@@std@@@std@@QBA_NABV012@@Z 00102c40 f i winmodemstat.obj
 0001:00001c88       ??E?$_Const_iterator@$00@?$list@VCResultListElement@@V?$allocator@VCResultListElement@@@std@@@std@@QAAAAV012@XZ 00102c88 f i winmodemstat.obj
 0001:00001cc4       ?_Inside@?$basic_string@DU?$char_traits@D@std@@V?$allocator@D@2@@std@@IAA_NPBD@Z 00102cc4 f i winmodemstat.obj
 0001:00001d04       ??$_Allocate@U_Node@?$_List_nod@VCResultListElement@@V?$allocator@VCResultListElement@@@std@@@std@@@std@@YAPAU_Node@?$_List_nod@VCResultListElement@@V?$allocator@VCResultListElement@@@std@@@0@IPAU120@@Z 00102d04 f i winmodemstat.obj
 0001:00001d74       ??$_Allocate@D@std@@YAPADIPAD@Z 00102d74 f i winmodemstat.obj
 0001:00001de0       ??0bad_alloc@std@@QAA@ABV01@@Z 00102de0 f i winmodemstat.obj
 0001:00001e00       ??1CModemStatus@@UAA@XZ    00102e00 f   winmodemstat.obj
 0001:00001e10       ??_ECModemStatus@@UAAPAXI@Z 00102e10 f i winmodemstat.obj
 0001:00001e10       ??_GCModemStatus@@UAAPAXI@Z 00102e10 f i winmodemstat.obj
 0001:00001e40       ?_Tidy@?$basic_string@DU?$char_traits@D@std@@V?$allocator@D@2@@std@@IAAX_NI@Z 00102e40 f i winmodemstat.obj
 0001:00001ea0       ?_Buynode@?$list@VCResultListElement@@V?$allocator@VCResultListElement@@@std@@@std@@IAAPAU_Node@?$_List_nod@VCResultListElement@@V?$allocator@VCResultListElement@@@std@@@2@XZ 00102ea0 f i winmodemstat.obj
 0001:00001ec4       ?erase@?$basic_string@DU?$char_traits@D@std@@V?$allocator@D@2@@std@@QAAAAV12@II@Z 00102ec4 f i winmodemstat.obj
 0001:00001f58       ?_Buynode@?$list@VCResultListElement@@V?$allocator@VCResultListElement@@@std@@@std@@IAAPAU_Node@?$_List_nod@VCResultListElement@@V?$allocator@VCResultListElement@@@std@@@2@PAU342@0ABVCResultListElement@@@Z 00102f58 f i winmodemstat.obj
 0001:00001fb8       ?_Copy@?$basic_string@DU?$char_traits@D@std@@V?$allocator@D@2@@std@@IAAXII@Z 00102fb8 f i winmodemstat.obj
 0001:00002100       ??1?$basic_string@DU?$char_traits@D@std@@V?$allocator@D@2@@std@@QAA@XZ 00103100 f i winmodemstat.obj
 0001:0000210c       ?_Grow@?$basic_string@DU?$char_traits@D@std@@V?$allocator@D@2@@std@@IAA_NI_N@Z 0010310c f i winmodemstat.obj
 0001:000021b0       ?clear@?$list@VCResultListElement@@V?$allocator@VCResultListElement@@@std@@@std@@QAAXXZ 001031b0 f i winmodemstat.obj
 0001:00002208       ??1logic_error@std@@UAA@XZ 00103208 f i winmodemstat.obj
 0001:00002234       ?what@logic_error@std@@UBAPBDXZ 00103234 f i winmodemstat.obj
 0001:0000224c       ??_Elogic_error@std@@UAAPAXI@Z 0010324c f i winmodemstat.obj
 0001:0000224c       ??_Glogic_error@std@@UAAPAXI@Z 0010324c f i winmodemstat.obj
 0001:0000228c       ?erase@?$list@VCResultListElement@@V?$allocator@VCResultListElement@@@std@@@std@@QAA?AV?$_Iterator@$00@12@V312@@Z 0010328c f i winmodemstat.obj
 0001:0000231c       ?assign@?$basic_string@DU?$char_traits@D@std@@V?$allocator@D@2@@std@@QAAAAV12@ABV12@II@Z 0010331c f i winmodemstat.obj
 0001:000023e0       ?assign@?$basic_string@DU?$char_traits@D@std@@V?$allocator@D@2@@std@@QAAAAV12@PBDI@Z 001033e0 f i winmodemstat.obj
 0001:00002488       ?RilResultCallback@CModemStatus@@KAXKJPBXKK@Z 00103488 f   winmodemstat.obj
 0001:00002864       ??0logic_error@std@@QAA@ABV?$basic_string@DU?$char_traits@D@std@@V?$allocator@D@2@@1@@Z 00103864 f i winmodemstat.obj
 0001:000028dc       ??1length_error@std@@UAA@XZ 001038dc f i winmodemstat.obj
 0001:00002908       ??_Glength_error@std@@UAAPAXI@Z 00103908 f i winmodemstat.obj
 0001:00002908       ??_Elength_error@std@@UAAPAXI@Z 00103908 f i winmodemstat.obj
 0001:00002948       ??0?$basic_string@DU?$char_traits@D@std@@V?$allocator@D@2@@std@@QAA@PBD@Z 00103948 f i winmodemstat.obj
 0001:00002988       ?_Incsize@?$list@VCResultListElement@@V?$allocator@VCResultListElement@@@std@@@std@@IAAXI@Z 00103988 f i winmodemstat.obj
 0001:00002a38       ??0logic_error@std@@QAA@ABV01@@Z 00103a38 f i winmodemstat.obj
 0001:00002ab0       ??0length_error@std@@QAA@ABV01@@Z 00103ab0 f i winmodemstat.obj
 0001:00002ad0       ?insert@?$list@VCResultListElement@@V?$allocator@VCResultListElement@@@std@@@std@@QAA?AV?$_Iterator@$00@12@V312@ABVCResultListElement@@@Z 00103ad0 f i winmodemstat.obj
 0001:00002b4c       ?AddResultItem@CModemStatus@@KAXJW4eFuncId@CResultListElement@@K@Z 00103b4c f   winmodemstat.obj
 0001:00002c58       ?ModGetOpState@CModemStatus@@SAJXZ 00103c58 f   winmodemstat.obj
 0001:00002c90       ?ModGetCallList@CModemStatus@@SAJXZ 00103c90 f   winmodemstat.obj
 0001:00002dc4       ?ModGetRegistrationStatus@CModemStatus@@SAJXZ 00103dc4 f   winmodemstat.obj
 0001:00002f00       ?RilNotifyCallback@CModemStatus@@KAXKPBXKK@Z 00103f00 f   winmodemstat.obj
 0001:000032f0       ?PowerSaveExit@CModemStatus@@SAXXZ 001042f0 f   winmodemstat.obj
 0001:00003338       ?ModSetEquipmentState@CModemStatus@@SAJK@Z 00104338 f   winmodemstat.obj
 0001:000034b4       ?HangUp@CModemStatus@@SAJXZ 001044b4 f   winmodemstat.obj
 0001:000035d8       ?Init@CModemStatus@@QAAJPAUHWND__@@@Z 001045d8 f   winmodemstat.obj
 0001:0000367c       RIL_Deinitialize           0010467c f   ril:ril.dll
 0001:0000368c       RIL_GetEquipmentState      0010468c f   ril:ril.dll
 0001:0000369c       RIL_GetCallList            0010469c f   ril:ril.dll
 0001:000036ac       RIL_GetRegistrationStatus  001046ac f   ril:ril.dll
 0001:000036bc       RIL_DevSpecific            001046bc f   ril:ril.dll
 0001:000036cc       RIL_SetEquipmentState      001046cc f   ril:ril.dll
 0001:000036dc       RIL_Hangup                 001046dc f   ril:ril.dll
 0001:000036ec       RIL_Initialize             001046ec f   ril:ril.dll
 0001:000036fc       tapiRequestMakeCallW       001046fc f   Cellcore:cellcore.dll
 0001:0000370c       SHGetEmergencyCallList     0010470c f   aygshell:AYGSHELL.dll
 0001:0000371c       PhoneMakeCall              0010471c f   phone:PHONE.dll
 0001:0000372c       ??3@YAXPAX@Z               0010472c f   coredll:COREDLL.dll
 0001:0000373c       ??2@YAPAXI@Z               0010473c f   coredll:COREDLL.dll
 0001:0000374c       memcmp                     0010474c f   coredll:COREDLL.dll
 0001:0000375c       wcsrchr                    0010475c f   coredll:COREDLL.dll
 0001:0000376c       CreateProcessW             0010476c f   coredll:COREDLL.dll
 0001:0000377c       CreateWindowExW            0010477c f   coredll:COREDLL.dll
 0001:0000378c       GetLastError               0010478c f   coredll:COREDLL.dll
 0001:0000379c       RegisterClassW             0010479c f   coredll:COREDLL.dll
 0001:000037ac       swprintf                   001047ac f   coredll:COREDLL.dll
 0001:000037bc       GetStockObject             001047bc f   coredll:COREDLL.dll
 0001:000037cc       memset                     001047cc f   coredll:COREDLL.dll
 0001:000037dc       DestroyWindow              001047dc f   coredll:COREDLL.dll
 0001:000037ec       wcscmp                     001047ec f   coredll:COREDLL.dll
 0001:000037fc       wcscpy                     001047fc f   coredll:COREDLL.dll
 0001:0000380c       MessageBoxW                0010480c f   coredll:COREDLL.dll
 0001:0000381c       LoadStringW                0010481c f   coredll:COREDLL.dll
 0001:0000382c       Sleep                      0010482c f   coredll:COREDLL.dll
 0001:0000383c       InsertMenuW                0010483c f   coredll:COREDLL.dll
 0001:0000384c       wcslen                     0010484c f   coredll:COREDLL.dll
 0001:0000385c       _purecall                  0010485c f   coredll:COREDLL.dll
 0001:0000386c       RaiseException             0010486c f   coredll:COREDLL.dll
 0001:0000387c       InitializeCriticalSection  0010487c f   coredll:COREDLL.dll
 0001:0000388c       __C_specific_handler       0010488c f   coredll:COREDLL.dll
 0001:0000389c       DeleteCriticalSection      0010489c f   coredll:COREDLL.dll
 0001:000038ac       free                       001048ac f   coredll:COREDLL.dll
 0001:000038bc       EventModify                001048bc f   coredll:COREDLL.dll
 0001:000038cc       strlen                     001048cc f   coredll:COREDLL.dll
 0001:000038dc       ??0exception@std@@QAA@PBD@Z 001048dc f   coredll:COREDLL.dll
 0001:000038ec       ?what@exception@std@@UBAPBDXZ 001048ec f   coredll:COREDLL.dll
 0001:000038fc       ??1exception@std@@UAA@XZ   001048fc f   coredll:COREDLL.dll
 0001:0000390c       CreateEventW               0010490c f   coredll:COREDLL.dll
 0001:0000391c       SendMessageTimeout         0010491c f   coredll:COREDLL.dll
 0001:0000392c       memcpy                     0010492c f   coredll:COREDLL.dll
 0001:0000393c       __CxxThrowException        0010493c f   coredll:COREDLL.dll
 0001:0000394c       ??_7type_info@@6B@         0010494c f   coredll:COREDLL.dll
 0001:0000395c       ??0exception@std@@QAA@ABV01@@Z 0010495c f   coredll:COREDLL.dll
 0001:0000396c       ??0exception@std@@QAA@XZ   0010496c f   coredll:COREDLL.dll
 0001:0000397c       TerminateProcess           0010497c f   coredll:COREDLL.dll
 0001:0000398c       PostMessageW               0010498c f   coredll:COREDLL.dll
 0001:0000399c       _DllMainCRTStartup         0010499c f   corelibc:pegdmain.obj
 0001:00003a34       __security_check_cookie    00104a34     corelibc:armsecgs.obj
 0001:00003a48       __gsfailure                00104a48     corelibc:armsecgs.obj
 0001:00003a8c       _onexit                    00104a8c f   corelibc:onexit.obj
 0001:00003b38       atexit                     00104b38 f   corelibc:onexit.obj
 0001:00003b58       _cinit                     00104b58 f   corelibc:crt0dat.obj
 0001:00003cc8       _cexit                     00104cc8 f   corelibc:crt0dat.obj
 0001:00003ce4       __security_init_cookie     00104ce4 f   corelibc:seccinit.obj
 0001:00003d3c       __FrameUnwindToState       00104d3c f   LIBCMT:frame_ce.obj
 0001:000040b4       ?_DestructExceptionObject@@YAXPAUEHExceptionRecord@@E@Z 001050b4 f   LIBCMT:frame_ce.obj
 0001:00004120       ?_OffsetToAddress@@YAPAXHPAKK@Z 00105120 f   LIBCMT:frame_ce.obj
 0001:0000416c       ?FindFrameInfo@@YAPAU_FrameInfo@@PAK@Z 0010516c f   LIBCMT:frame_ce.obj
 0001:000041ac       ?FindCatchFrameInfo@@YAPAU_FrameInfo@@PAK@Z 001051ac f   LIBCMT:frame_ce.obj
 0001:000041ec       ?_GetRangeOfTrysToCheck@@YAPBU_s_TryBlockMapEntry@@PBU_s_FuncInfo@@HHPAI1@Z 001051ec f   LIBCMT:frame_ce.obj
 0001:00004bf8       __InternalCxxFrameHandler  00105bf8 f   LIBCMT:frame_ce.obj
 0001:00004d50       __CxxFrameHandler3         00105d50 f   LIBCMT:frame_ce.obj
 0001:00004d88       __GSHandlerCheckCommon     00105d88 f   LIBCMT:gshandler.obj
 0001:00004dd0       __GSHandlerCheck           00105dd0 f   LIBCMT:gshandler.obj
 0001:00004e00       memcpy_s                   00105e00 f   LIBCMT:memcpy_s.obj
 0001:00004ee8       memmove_s                  00105ee8 f   LIBCMT:memmove_s.obj
 0001:00004fa0       _invalid_parameter_noinfo  00105fa0 f   LIBCMT:invarg.obj
 0001:00004fdc       _invoke_watson             00105fdc f   LIBCMT:invarg.obj
 0001:00005008       __GSHandlerCheck_EH        00106008 f   LIBCMT:gshandlereh.obj
 0001:0000509c       GetCRTStorage              0010609c f   LIBCMT:corecrt.obj
 0001:00005168       _CallSettingFrame          00106168     LIBCMT:handlers_arm.obj
 0001:000051ac       ?FindFrameForUnwind@@YAPAKPAKPBU_s_FuncInfo@@@Z 001061ac f   LIBCMT:mdframe_arm.obj
 0001:000051f4       ?FindCatchFrame@@YAPAKPAKK@Z 001061f4 f   LIBCMT:mdframe_arm.obj
 0001:00005240       ?AdjustFrameForCatch@@YAPAKPAKPBU_s_FuncInfo@@@Z 00106240 f   LIBCMT:mdframe_arm.obj
 0001:00005278       ?GetCurrentState@@YAHPAKPAU_DISPATCHER_CONTEXT@@PBU_s_FuncInfo@@@Z 00106278 f   LIBCMT:ehstate_arm_mips.obj
 0001:000052d4       _invalid_parameter         001062d4 f   LIBCMT:invarginternal.obj
 0001:00005300       ??1out_of_range@std@@UAA@XZ 00106300 f i libcpmt:string.obj
 0001:0000532c       ??_Gout_of_range@std@@UAAPAXI@Z 0010632c f i libcpmt:string.obj
 0001:0000532c       ??_Eout_of_range@std@@UAAPAXI@Z 0010632c f i libcpmt:string.obj
 0001:00005380       ?_Xlen@_String_base@std@@SAXXZ 00106380 f   libcpmt:string.obj
 0001:00005410       ?_Xran@_String_base@std@@SAXXZ 00106410 f   libcpmt:string.obj
 0001:00005498       ??0out_of_range@std@@QAA@ABV01@@Z 00106498 f i libcpmt:string.obj
 0001:000054c8       AtlRawDllMain              001064c8 f   atls:atlbase.obj
 0001:00005560       ?RemoveAll@?$CSimpleArray@PAUHINSTANCE__@@V?$CSimpleArrayEqualHelper@PAUHINSTANCE__@@@ATL@@@ATL@@QAAXXZ 00106560 f i atls:atlbase.obj
 0001:0000559c       ??0_ATL_BASE_MODULE70@ATL@@QAA@XZ 0010659c f i atls:atlbase.obj
 0001:000055e0       ??1CAtlBaseModule@ATL@@QAA@XZ 001065e0 f   atls:atlbase.obj
 0001:00005618       ??0CAtlBaseModule@ATL@@QAA@XZ 00106618 f   atls:atlbase.obj
 0001:000056b4       __report_gsfailure         001066b4 f   coredll:COREDLL.dll
 0001:000056c4       LocalReAlloc               001066c4 f   coredll:COREDLL.dll
 0001:000056d4       LocalAlloc                 001066d4 f   coredll:COREDLL.dll
 0001:000056e4       LocalSize                  001066e4 f   coredll:COREDLL.dll
 0001:000056f4       LocalFree                  001066f4 f   coredll:COREDLL.dll
 0001:00005704       __security_gen_cookie      00106704 f   coredll:COREDLL.dll
 0001:00005714       strcmp                     00106714 f   coredll:COREDLL.dll
 0001:00005724       ?terminate@std@@YAXXZ      00106724 f   coredll:COREDLL.dll
 0001:00005734       memmove                    00106734 f   coredll:COREDLL.dll
 0001:00005744       TlsCall                    00106744 f   coredll:COREDLL.dll
 0001:00005754       TlsSetValue                00106754 f   coredll:COREDLL.dll
 0001:00005764       TlsGetValue                00106764 f   coredll:COREDLL.dll
 0001:00005774       InterlockedCompareExchange 00106774 f   coredll:COREDLL.dll
 0001:00005784       GetModuleHandleW           00106784 f   coredll:COREDLL.dll
 0002:00000000       ??_7CSWContextMenuClassFactory@@6B@ 00107000     clsfact.obj
 0002:00000070       ??_C@_15LCCIEICG@?$AA?$CK?$AA2?$AA?$AA@ 00107070     DialParsExtOEM.obj
 0002:00000078       ??_C@_19KFCMCMMA@?$AA?$CD?$AA9?$AA1?$AA1?$AA?$AA@ 00107078     DialParsExtOEM.obj
 0002:00000084       ??_C@_19FJDJAHAK@?$AA?$CK?$AA9?$AA1?$AA1?$AA?$AA@ 00107084     DialParsExtOEM.obj
 0002:00000090       ??_C@_17IHOOCDAM@?$AA9?$AA1?$AA1?$AA?$AA@ 00107090     DialParsExtOEM.obj
 0002:00000098       ??_C@_0P@GHFPNOJB@bad?5allocation?$AA@ 00107098     DialParsExtOEM.obj
 0002:000000a8       CLSID_ShellDesktop         001070a8     DialParsExtOEM.obj
 0002:000000b8       IID_IContextMenu           001070b8     DialParsExtOEM.obj
 0002:000000c8       IID_IShellFolder           001070c8     DialParsExtOEM.obj
 0002:000000d8       IID_IShellExtInit          001070d8     DialParsExtOEM.obj
 0002:000000e8       IID_IShellPropSheetExt     001070e8     DialParsExtOEM.obj
 0002:000000f8       IID_IEnumIDList            001070f8     DialParsExtOEM.obj
 0002:00000108       IID_IShellCommandUI        00107108     DialParsExtOEM.obj
 0002:00000118       IID_IShellListView         00107118     DialParsExtOEM.obj
 0002:00000128       IID_IShellFind             00107128     DialParsExtOEM.obj
 0002:00000138       IID_IShellFindItem         00107138     DialParsExtOEM.obj
 0002:00000148       IID_IShellFindCallback     00107148     DialParsExtOEM.obj
 0002:00000158       IID_IShellNotificationCallback 00107158     DialParsExtOEM.obj
 0002:00000168       IID_INewMenuItemServer     00107168     DialParsExtOEM.obj
 0002:00000178       IID_IAutoSuggestionGenerator 00107178     DialParsExtOEM.obj
 0002:00000188       CLSID_CSWContextMenu       00107188     DialParsExtOEM.obj
 0002:000001cc       ??_C@_1DO@GKGCGOMO@?$AAM?$AAo?$AAd?$AAe?$AAm?$AAS?$AAt?$AAa?$AAt?$AA?5?$AAI?$AAn?$AAi?$AAt?$AAi?$AAa?$AAl?$AAi?$AAz?$AAe?$AA?5?$AAF?$AAa?$AAi?$AAl?$AAe?$AAd?$AA?5?$AA?$CF?$AAd?$AA?$AA@ 001071cc     DialParsExtOEM.obj
 0002:0000020c       ??_C@_1DG@EIKBGNDO@?$AAg?$AAh?$AAw?$AAn?$AAd?$AAR?$AAi?$AAl?$AAM?$AAe?$AAs?$AAs?$AAa?$AAg?$AAe?$AA?5?$AAs?$AAt?$AAi?$AAl?$AAl?$AA?5?$AAN?$AAU?$AAL?$AAL?$AA?$AA@ 0010720c     DialParsExtOEM.obj
 0002:00000244       ??_C@_1CK@PIKJOKFL@?$AA?4?$AA?2?$AAD?$AAi?$AAa?$AAl?$AAP?$AAa?$AAr?$AAs?$AAE?$AAx?$AAt?$AAO?$AAE?$AAM?$AA?4?$AAc?$AAp?$AAp?$AA?$AA@ 00107244     DialParsExtOEM.obj
 0002:00000270       ??_C@_1DA@HAPCEKP@?$AAU?$AAn?$AAa?$AAb?$AAl?$AAe?$AA?5?$AAt?$AAo?$AA?5?$AAL?$AAa?$AAu?$AAn?$AAc?$AAh?$AAR?$AAi?$AAl?$AAt?$AAe?$AAs?$AAt?$AA?$AA@ 00107270     DialParsExtOEM.obj
 0002:000002a0       ??_C@_1CK@CFPCLIFE@?$AA?2?$AAW?$AAi?$AAn?$AAd?$AAo?$AAw?$AAs?$AA?2?$AAr?$AAi?$AAl?$AAt?$AAe?$AAs?$AAt?$AA?4?$AAe?$AAx?$AAe?$AA?$AA@ 001072a0     DialParsExtOEM.obj
 0002:000002cc       ??_C@_1DA@LFLONJOJ@?$AAU?$AAn?$AAa?$AAb?$AAl?$AAe?$AA?5?$AAt?$AAo?$AA?5?$AAL?$AAa?$AAu?$AAn?$AAc?$AAh?$AAR?$AAe?$AAg?$AAE?$AAd?$AAi?$AAt?$AA?$AA@ 001072cc     DialParsExtOEM.obj
 0002:000002fc       ??_C@_1CK@CJHOALLD@?$AA?2?$AAW?$AAi?$AAn?$AAd?$AAo?$AAw?$AAs?$AA?2?$AAr?$AAe?$AAg?$AAe?$AAd?$AAi?$AAt?$AA?4?$AAe?$AAx?$AAe?$AA?$AA@ 001072fc     DialParsExtOEM.obj
 0002:00000328       ??_C@_1EG@BKKBJIIL@?$AAU?$AAn?$AAa?$AAb?$AAl?$AAe?$AA?5?$AAt?$AAo?$AA?5?$AAL?$AAa?$AAu?$AAn?$AAc?$AAh?$AA?5?$AAp?$AAh?$AAo?$AAn?$AAe?$AAu?$AAt?$AAi?$AAl?$AAi?$AAt?$AAy?$AAG?$AA?4?$AAe@ 00107328     DialParsExtOEM.obj
 0002:00000370       ??_C@_1DG@OJCDBIGD@?$AA?2?$AAW?$AAi?$AAn?$AAd?$AAo?$AAw?$AAs?$AA?2?$AAp?$AAh?$AAo?$AAn?$AAe?$AAu?$AAt?$AAi?$AAl?$AAi?$AAt?$AAy?$AAG?$AA?4?$AAe?$AAx?$AAe?$AA?$AA@ 00107370     DialParsExtOEM.obj
 0002:000003a8       ??_C@_1EC@CLLBLAAJ@?$AAF?$AAa?$AAi?$AAl?$AA?5?$AAt?$AAo?$AA?5?$AAC?$AAr?$AAe?$AAa?$AAt?$AAe?$AAW?$AAi?$AAn?$AAd?$AAo?$AAw?$AA?0?$AA?5?$AAe?$AAr?$AAr?$AA?5?$AA?$DN?$AA?5?$AA0?$AAx?$AA?$CF?$AAx@ 001073a8     DialParsExtOEM.obj
 0002:000003ec       ??_C@_1DC@EDDBJNIM@?$AAC?$AAS?$AAW?$AA_?$AAD?$AAi?$AAa?$AAl?$AAP?$AAa?$AAr?$AAs?$AAe?$AAr?$AAM?$AAs?$AAg?$AAC?$AAl?$AAa?$AAs?$AAs?$AA?$CF?$AAx?$AA?$AA@ 001073ec     DialParsExtOEM.obj
 0002:00000420       ??_C@_1GM@IHMNDCIB@?$AAS?$AAW?$AAD?$AAi?$AAa?$AAl?$AAP?$AAa?$AAr?$AAs?$AAe?$AAr?$AA?5?$AAD?$AAl?$AAl?$AAM?$AAa?$AAi?$AAn?$AA?5?$AAe?$AAx?$AAi?$AAt?$AA?5?$AAb?$AAc?$AAo?$AAs?$AA?5?$AAg@ 00107420     DialParsExtOEM.obj
 0002:0000048c       ??_C@_1BE@OIBEOKIJ@?$AAR?$AAo?$AAa?$AAm?$AAG?$AAu?$AAa?$AAr?$AAd?$AA?$AA@ 0010748c     DialParsExtOEM.obj
 0002:000004a0       ??_C@_1O@GINMMDNN@?$AAS?$AAy?$AAs?$AAt?$AAe?$AAm?$AA?$AA@ 001074a0     DialParsExtOEM.obj
 0002:000004b0       ??_7Csw_ctxMenu@@6BIContextMenu@@@ 001074b0     DialParsExtOEM.obj
 0002:000004c8       ??_7Csw_ctxMenu@@6BIObjectWithSite@@@ 001074c8     DialParsExtOEM.obj
 0002:000004dc       ??_C@_1BK@EFKFIHCE@?$AAP?$AAh?$AAo?$AAn?$AAe?$AA?5?$AAD?$AAi?$AAa?$AAl?$AAe?$AAr?$AA?$AA@ 001074dc     DialParsExtOEM.obj
 0002:000004f8       ??_C@_1EG@HGDDPKED@?$AAU?$AAn?$AAa?$AAb?$AAl?$AAe?$AA?5?$AAt?$AAo?$AA?5?$AAL?$AAa?$AAu?$AAn?$AAc?$AAh?$AA?5?$AAA?$AAc?$AAt?$AAi?$AAv?$AAa?$AAt?$AAi?$AAo?$AAn?$AA?5?$AAW?$AAi?$AAz?$AAa@ 001074f8     DialParsExtOEM.obj
 0002:00000540       ??_C@_1DI@LFPNANLM@?$AA?2?$AAW?$AAi?$AAn?$AAd?$AAo?$AAw?$AAs?$AA?2?$AAG?$AAo?$AAb?$AAi?$AAa?$AAc?$AAt?$AAi?$AAv?$AAa?$AAt?$AAi?$AAo?$AAn?$AA?4?$AAe?$AAx?$AAe?$AA?$AA@ 00107540     DialParsExtOEM.obj
 0002:00000578       ??_C@_13GMDMCADD@?$AA?$CD?$AA?$AA@ 00107578     DialParsExtOEM.obj
 0002:0000057c       ??_C@_15HNICCJBE@?$AA?$CD?$AA?$CD?$AA?$AA@ 0010757c     DialParsExtOEM.obj
 0002:00000584       ??_C@_1BE@KLOIBIOC@?$AA?$CD?$AA?$CD?$AAr?$AAi?$AAl?$AAt?$AAe?$AAs?$AAt?$AA?$AA@ 00107584     DialParsExtOEM.obj
 0002:00000598       ??_C@_1BE@JMCIFKMF@?$AA?$CD?$AA?$CD?$AA7?$AA4?$AA5?$AA8?$AA3?$AA7?$AA8?$AA?$AA@ 00107598     DialParsExtOEM.obj
 0002:000005ac       ??_C@_1BE@FGAEOGHE@?$AA?$CD?$AA?$CD?$AAr?$AAe?$AAg?$AAe?$AAd?$AAi?$AAt?$AA?$AA@ 001075ac     DialParsExtOEM.obj
 0002:000005c0       ??_C@_1BE@BMDEDFDD@?$AA?$CD?$AA?$CD?$AA7?$AA3?$AA4?$AA3?$AA3?$AA4?$AA8?$AA?$AA@ 001075c0     DialParsExtOEM.obj
 0002:000005d4       ??_C@_1M@EBALFFOP@?$AA?$CD?$AA?$CD?$AAa?$AAw?$AAz?$AA?$AA@ 001075d4     DialParsExtOEM.obj
 0002:000005e0       ??_C@_1M@CGFBDNAF@?$AA?$CD?$AA?$CD?$AA2?$AA9?$AA9?$AA?$AA@ 001075e0     DialParsExtOEM.obj
 0002:000005ec       ??_7IObjectWithSite@@6B@   001075ec     DialParsExtOEM.obj
 0002:00000600       ??_C@_1KK@BFBKODDO@?$AAP?$AAr?$AAe?$AAp?$AAr?$AAo?$AAc?$AAe?$AAs?$AAs?$AAD?$AAi?$AAa?$AAl?$AAR?$AAe?$AAq?$AAu?$AAe?$AAs?$AAt?$AA?9?$AA?$DO?$AAC?$AAr?$AAe?$AAa?$AAt?$AAe?$AAM?$AAe?$AAs@ 00107600     DialParsExtOEM.obj
 0002:000006b0       ??_C@_1JM@EKIHANIH@?$AAD?$AAi?$AAa?$AAl?$AA?5?$AAr?$AAe?$AAq?$AAu?$AAe?$AAs?$AAt?$AA?5?$AAr?$AAe?$AAj?$AAe?$AAc?$AAt?$AAe?$AAd?$AA?5?$AAb?$AAy?$AA?5?$AAP?$AAh?$AAo?$AAn?$AAe?$AAM?$AAa@ 001076b0     DialParsExtOEM.obj
 0002:00000750       ??_C@_1GM@PLKCGKGJ@?$AAs?$AAp?$AAe?$AAc?$AAi?$AAa?$AAl?$AA?5?$AAE?$AAn?$AAd?$AA?5?$AAC?$AAa?$AAl?$AAl?$AA?5?$AAc?$AAo?$AAm?$AAm?$AAa?$AAn?$AAd?$AA?5?$AAr?$AAe?$AAc?$AAe?$AAi?$AAv?$AAe@ 00107750     DialParsExtOEM.obj
 0002:000007bc       ??_C@_17KBCCMHPH@?$AA3?$AA6?$AA3?$AA?$AA@ 001077bc     DialParsExtOEM.obj
 0002:000007c8       ??_C@_1JG@HAAEOLCE@?$AAC?$AAs?$AAw?$AA_?$AAc?$AAt?$AAx?$AAM?$AAe?$AAn?$AAu?$AA?9?$AA?$DO?$AAC?$AAr?$AAe?$AAa?$AAt?$AAe?$AAM?$AAe?$AAs?$AAs?$AAa?$AAg?$AAe?$AAW?$AAi?$AAn?$AAd?$AAo?$AAw@ 001077c8     DialParsExtOEM.obj
 0002:00000860       ??_C@_1O@JDLOHAN@?$AAD?$AAe?$AAl?$AAe?$AAt?$AAe?$AA?$AA@ 00107860     resultelement.obj
 0002:00000870       ??_C@_1BC@GCKHIPE@?$AAN?$AAo?$AAR?$AAe?$AAm?$AAo?$AAv?$AAe?$AA?$AA@ 00107870     resultelement.obj
 0002:00000884       ??_C@_1BI@JFAIJMHL@?$AAF?$AAo?$AAr?$AAc?$AAe?$AAR?$AAe?$AAm?$AAo?$AAv?$AAe?$AA?$AA@ 00107884     resultelement.obj
 0002:0000089c       ??_C@_17LLMMEOJD@?$AAV?$AAa?$AAl?$AA?$AA@ 0010789c     resultelement.obj
 0002:000008a4       ??_C@_13OPKGLAFF@?$AAB?$AA?$AA@ 001078a4     resultelement.obj
 0002:000008a8       ??_C@_13MKMNOPIJ@?$AAD?$AA?$AA@ 001078a8     resultelement.obj
 0002:000008ac       ??_C@_13LHMFKAAD@?$AAM?$AA?$AA@ 001078ac     resultelement.obj
 0002:000008b0       ??_C@_13HADIAKP@?$AAS?$AA?$AA@ 001078b0     resultelement.obj
 0002:000008d4       ??_7CResultListElement@@6B@ 001078d4     resultelement.obj
 0002:000008f8       ??_7CModemStatus@@6B@      001078f8     winmodemstat.obj
 0002:000008fc       ??_C@_1CG@IOFFODIG@?$AAM?$AAO?$AAD?$AAE?$AAM?$AA_?$AAO?$AAN?$AA_?$AAO?$AAF?$AAF?$AA_?$AAE?$AAV?$AAE?$AAN?$AAT?$AA?$AA@ 001078fc     winmodemstat.obj
 0002:00000928       ??_C@_1FI@HMJKAGBH@?$AA?4?$AA?4?$AA?2?$AA?4?$AA?4?$AA?2?$AAR?$AAI?$AAL?$AAD?$AAr?$AAi?$AAv?$AAe?$AAr?$AA?2?$AAC?$AAo?$AAm?$AAm?$AAo?$AAn?$AA?2?$AAs?$AAr?$AAc?$AA?2?$AAw?$AAi?$AAn?$AAm?$AAo@ 00107928     winmodemstat.obj
 0002:00000980       ??_C@_1JO@DKICHNLH@?$AAS?$AAe?$AAn?$AAd?$AA?5?$AAm?$AAe?$AAs?$AAs?$AAa?$AAg?$AAe?$AA?5?$AAt?$AAi?$AAm?$AAe?$AAo?$AAu?$AAt?$AA?5?$AAf?$AAr?$AAo?$AAm?$AA?5?$AAw?$AAi?$AAn?$AAm?$AAo?$AAd@ 00107980     winmodemstat.obj
 0002:00000a20       ??_C@_1GG@MLOAOBHO@?$AAU?$AAp?$AAd?$AAa?$AAt?$AAe?$AAC?$AAa?$AAl?$AAl?$AAT?$AAy?$AAp?$AAe?$AAA?$AAn?$AAd?$AAS?$AAt?$AAa?$AAt?$AAu?$AAs?$AA?5?$AAc?$AAa?$AAn?$AAn?$AAo?$AAt?$AA?5?$AAh@ 00107a20     winmodemstat.obj
 0002:00000a88       ??_C@_1JG@JMBAMLCB@?$AAI?$AAn?$AAv?$AAa?$AAl?$AAi?$AAd?$AA?5?$AAs?$AAt?$AAa?$AAt?$AAe?$AA?3?$AA?5?$AAm?$AA_?$AAC?$AAa?$AAl?$AAl?$AAT?$AAy?$AAp?$AAe?$AA?5?$AA?$DN?$AA?5?$AA?$CF?$AAd?$AA?5?$AAb@ 00107a88     winmodemstat.obj
 0002:00000b20       ??_C@_1FO@GFODOKOF@?$AAI?$AAn?$AAv?$AAa?$AAl?$AAi?$AAd?$AA?5?$AAs?$AAt?$AAa?$AAt?$AAe?$AA?3?$AA?5?$AAm?$AA_?$AAC?$AAa?$AAl?$AAl?$AAT?$AAy?$AAp?$AAe?$AA?5?$AA?$DN?$AA?5?$AA?$CF?$AAd?$AA?5?$AAb@ 00107b20     winmodemstat.obj
 0002:00000b80       ??_C@_1DK@CMAHCKEF@?$AAI?$AAn?$AAv?$AAa?$AAl?$AAi?$AAd?$AA?5?$AAc?$AAa?$AAl?$AAl?$AAE?$AAv?$AAe?$AAn?$AAt?$AAM?$AAa?$AAs?$AAk?$AA?5?$AA?$DN?$AA?5?$AA0?$AAx?$AA?$CF?$AAx?$AA?$AA@ 00107b80     winmodemstat.obj
 0002:00000bbc       ??_C@_1CI@CHFKALHP@?$AAU?$AAN?$AAC?$AAH?$AAG?$AA?0?$AA?5?$AAi?$AAn?$AAv?$AAa?$AAl?$AAi?$AAd?$AA?5?$AAc?$AAa?$AAs?$AAe?$AA?$AA@ 00107bbc     winmodemstat.obj
 0002:00000d50       ??_C@_0BB@MOGOBHAF@list?$DMT?$DO?5too?5long?$AA@ 00107d50     winmodemstat.obj
 0002:00000df0       ??_C@_1NK@HKFOPGPM@?$AAI?$AAn?$AAv?$AAa?$AAl?$AAi?$AAd?$AA?5?$AAu?$AAs?$AAe?$AA?5?$AAo?$AAf?$AA?5?$AAA?$AAd?$AAd?$AAR?$AAe?$AAs?$AAu?$AAl?$AAt?$AAI?$AAt?$AAe?$AAm?$AA?5?$AAo?$AAn?$AA?5@ 00107df0     winmodemstat.obj
 0002:00000ed0       ??_C@_1GE@NCBFCKEM@?$AAA?$AAb?$AAo?$AAu?$AAt?$AA?5?$AAt?$AAo?$AA?5?$AAc?$AAa?$AAl?$AAl?$AA?5?$AAT?$AAe?$AAr?$AAm?$AAi?$AAn?$AAa?$AAt?$AAe?$AAP?$AAr?$AAo?$AAc?$AAe?$AAs?$AAs?$AA?5?$AAi@ 00107ed0     winmodemstat.obj
 0002:00000f38       ??_C@_1FC@IDFJCPGP@?$AAC?$AAA?$AAT?$AAC?$AAH?$AA_?$AAT?$AAH?$AAE?$AA_?$AAE?$AAR?$AAR?$AAO?$AAR?$AA?5?$AAb?$AAu?$AAt?$AA?5?$AAc?$AAa?$AAn?$AAn?$AAo?$AAt?$AA?5?$AAp?$AAo?$AAs?$AAt?$AA?5@ 00107f38     winmodemstat.obj
 0002:00001068       ??_C@_1FO@HEAAPBIE@?$AAC?$AAa?$AAr?$AAr?$AAi?$AAe?$AAr?$AA?5?$AAI?$AAn?$AAd?$AAe?$AAx?$AA?5?$AAC?$AAh?$AAn?$AAa?$AAg?$AAe?$AAd?$AA?5?$AAN?$AAO?$AAT?$AAI?$AAF?$AAY?$AA_?$AAC?$AAA?$AAR@ 00108068     winmodemstat.obj
 0002:000010c8       ??_C@_1DK@FPIKNIHL@?$AAR?$AAI?$AAL?$AA_?$AAN?$AAO?$AAT?$AAI?$AAF?$AAY?$AA_?$AAP?$AAD?$AAP?$AA_?$AAI?$AAN?$AAA?$AAC?$AAT?$AA_?$AAF?$AAA?$AAI?$AAL?$AA_?$AAE?$AA?5?$AA?$AA@ 001080c8     winmodemstat.obj
 0002:00001108       ??_C@_1KE@BGFKGAIL@?$AAT?$AAe?$AAl?$AAl?$AA?5?$AAo?$AAu?$AAr?$AA?5?$AAa?$AAp?$AAp?$AAs?$AA?5?$AAt?$AAo?$AA?5?$AAc?$AAl?$AAe?$AAa?$AAn?$AA?5?$AAu?$AAp?$AA?5?$AAt?$AAh?$AAe?$AA?5?$AAc?$AAa@ 00108108     winmodemstat.obj
 0002:00001288       ??_C@_1EK@PLMMIOKB@?$AAR?$AAI?$AAL?$AA_?$AAI?$AAn?$AAi?$AAt?$AAi?$AAa?$AAl?$AAi?$AAz?$AAe?$AA?5?$AAf?$AAa?$AAi?$AAl?$AAe?$AAd?$AA?5?$AAh?$AAR?$AAe?$AAs?$AAu?$AAl?$AAt?$AA?5?$AA?$DN?$AA?5@ 00108288     winmodemstat.obj
 0002:000012d4       IID_IClassFactory          001082d4     uuid:unknwn_i_guid1.obj
 0002:000012e4       IID_IUnknown               001082e4     uuid:unknwn_i_guid0.obj
 0002:000012f4       IID_IObjectWithSite        001082f4     uuid:ocidl_i_guid34.obj
 0002:00001308       ??_7bad_alloc@std@@6B@     00108308     libcpmt:string.obj
 0002:00001314       ??_7logic_error@std@@6B@   00108314     libcpmt:string.obj
 0002:00001320       ??_7length_error@std@@6B@  00108320     libcpmt:string.obj
 0002:0000132c       ??_7out_of_range@std@@6B@  0010832c     libcpmt:string.obj
 0002:00001380       ??_C@_0BA@JFNIOLAK@string?5too?5long?$AA@ 00108380     libcpmt:string.obj
 0002:000013dc       ??_C@_0BI@CFPLBAOH@invalid?5string?5position?$AA@ 001083dc     libcpmt:string.obj
 0002:000013f4       GUID_ATLVer30              001083f4     atls:atlbase.obj
 0002:00001404       GUID_ATLVer70              00108404     atls:atlbase.obj
 0002:00001414       IID_IPersistStream         00108414     uuid:objidl_i_guid12.obj
 0002:00001424       ??_R4bad_alloc@std@@6B@    00108424     libcpmt:string.obj
 0002:00001438       ??_R3bad_alloc@std@@8      00108438     libcpmt:string.obj
 0002:00001448       ??_R2bad_alloc@std@@8      00108448     libcpmt:string.obj
 0002:00001454       ??_R1A@?0A@EA@bad_alloc@std@@8 00108454     libcpmt:string.obj
 0002:00001470       ??_R1A@?0A@EA@exception@std@@8 00108470     libcpmt:string.obj
 0002:0000148c       ??_R3exception@std@@8      0010848c     libcpmt:string.obj
 0002:0000149c       ??_R2exception@std@@8      0010849c     libcpmt:string.obj
 0002:000014a4       ??_R4logic_error@std@@6B@  001084a4     libcpmt:string.obj
 0002:000014b8       ??_R3logic_error@std@@8    001084b8     libcpmt:string.obj
 0002:000014c8       ??_R2logic_error@std@@8    001084c8     libcpmt:string.obj
 0002:000014d4       ??_R1A@?0A@EA@logic_error@std@@8 001084d4     libcpmt:string.obj
 0002:000014f0       ??_R4length_error@std@@6B@ 001084f0     libcpmt:string.obj
 0002:00001504       ??_R3length_error@std@@8   00108504     libcpmt:string.obj
 0002:00001514       ??_R2length_error@std@@8   00108514     libcpmt:string.obj
 0002:00001524       ??_R1A@?0A@EA@length_error@std@@8 00108524     libcpmt:string.obj
 0002:00001540       ??_R4out_of_range@std@@6B@ 00108540     libcpmt:string.obj
 0002:00001554       ??_R3out_of_range@std@@8   00108554     libcpmt:string.obj
 0002:00001564       ??_R2out_of_range@std@@8   00108564     libcpmt:string.obj
 0002:00001574       ??_R1A@?0A@EA@out_of_range@std@@8 00108574     libcpmt:string.obj
 0002:00001620       _TI2?AVbad_alloc@std@@     00108620     winmodemstat.obj
 0002:00001630       _CTA2?AVbad_alloc@std@@    00108630     winmodemstat.obj
 0002:0000163c       _CT??_R0?AVbad_alloc@std@@@8??0bad_alloc@std@@QAA@ABV01@@Z12 0010863c     winmodemstat.obj
 0002:00001658       _CT??_R0?AVexception@std@@@8??0exception@std@@QAA@ABV01@@Z12 00108658     winmodemstat.obj
 0002:00001674       _TI3?AVlength_error@std@@  00108674     winmodemstat.obj
 0002:00001684       _CTA3?AVlength_error@std@@ 00108684     winmodemstat.obj
 0002:00001694       _CT??_R0?AVlength_error@std@@@8??0length_error@std@@QAA@ABV01@@Z40 00108694     winmodemstat.obj
 0002:000016b0       _CT??_R0?AVlogic_error@std@@@8??0logic_error@std@@QAA@ABV01@@Z40 001086b0     winmodemstat.obj
 0002:000016cc       _TI3?AVout_of_range@std@@  001086cc     libcpmt:string.obj
 0002:000016dc       _CTA3?AVout_of_range@std@@ 001086dc     libcpmt:string.obj
 0002:000016ec       _CT??_R0?AVout_of_range@std@@@8??0out_of_range@std@@QAA@ABV01@@Z40 001086ec     libcpmt:string.obj
 0002:00001708       __IMPORT_DESCRIPTOR_sw_utilityG 00108708     sw_utilityG:sw_utilityG.dll
 0002:0000171c       __IMPORT_DESCRIPTOR_ril    0010871c     ril:ril.dll
 0002:00001730       __IMPORT_DESCRIPTOR_cellcore 00108730     Cellcore:cellcore.dll
 0002:00001744       __IMPORT_DESCRIPTOR_AYGSHELL 00108744     aygshell:AYGSHELL.dll
 0002:00001758       __IMPORT_DESCRIPTOR_PHONE  00108758     phone:PHONE.dll
 0002:0000176c       __IMPORT_DESCRIPTOR_COREDLL 0010876c     coredll:COREDLL.dll
 0002:00001780       __NULL_IMPORT_DESCRIPTOR   00108780     sw_utilityG:sw_utilityG.dll
 0003:00000000       __imp_SHGetEmergencyCallList 00109000     aygshell:AYGSHELL.dll
 0003:00000004       \177AYGSHELL_NULL_THUNK_DATA 00109004     aygshell:AYGSHELL.dll
 0003:00000008       __imp_GetModuleHandleW     00109008     coredll:COREDLL.dll
 0003:0000000c       __imp_InterlockedCompareExchange 0010900c     coredll:COREDLL.dll
 0003:00000010       __imp_TlsGetValue          00109010     coredll:COREDLL.dll
 0003:00000014       __imp___report_gsfailure   00109014     coredll:COREDLL.dll
 0003:00000018       __imp_TlsCall              00109018     coredll:COREDLL.dll
 0003:0000001c       __imp_memmove              0010901c     coredll:COREDLL.dll
 0003:00000020       __imp_?terminate@std@@YAXXZ 00109020     coredll:COREDLL.dll
 0003:00000024       __imp_strcmp               00109024     coredll:COREDLL.dll
 0003:00000028       __imp___security_gen_cookie 00109028     coredll:COREDLL.dll
 0003:0000002c       __imp_LocalFree            0010902c     coredll:COREDLL.dll
 0003:00000030       __imp_LocalSize            00109030     coredll:COREDLL.dll
 0003:00000034       __imp_LocalAlloc           00109034     coredll:COREDLL.dll
 0003:00000038       __imp_PostMessageW         00109038     coredll:COREDLL.dll
 0003:0000003c       __imp_TerminateProcess     0010903c     coredll:COREDLL.dll
 0003:00000040       __imp_TlsSetValue          00109040     coredll:COREDLL.dll
 0003:00000044       __imp_InitializeCriticalSection 00109044     coredll:COREDLL.dll
 0003:00000048       __imp_??0exception@std@@QAA@XZ 00109048     coredll:COREDLL.dll
 0003:0000004c       __imp_??3@YAXPAX@Z         0010904c     coredll:COREDLL.dll
 0003:00000050       __imp_??2@YAPAXI@Z         00109050     coredll:COREDLL.dll
 0003:00000054       __imp_memcmp               00109054     coredll:COREDLL.dll
 0003:00000058       __imp_wcsrchr              00109058     coredll:COREDLL.dll
 0003:0000005c       __imp_CreateProcessW       0010905c     coredll:COREDLL.dll
 0003:00000060       __imp_CreateWindowExW      00109060     coredll:COREDLL.dll
 0003:00000064       __imp_GetLastError         00109064     coredll:COREDLL.dll
 0003:00000068       __imp_RegisterClassW       00109068     coredll:COREDLL.dll
 0003:0000006c       __imp_swprintf             0010906c     coredll:COREDLL.dll
 0003:00000070       __imp_GetStockObject       00109070     coredll:COREDLL.dll
 0003:00000074       __imp_memset               00109074     coredll:COREDLL.dll
 0003:00000078       __imp_DestroyWindow        00109078     coredll:COREDLL.dll
 0003:0000007c       __imp_wcscmp               0010907c     coredll:COREDLL.dll
 0003:00000080       __imp_wcscpy               00109080     coredll:COREDLL.dll
 0003:00000084       __imp_MessageBoxW          00109084     coredll:COREDLL.dll
 0003:00000088       __imp_LoadStringW          00109088     coredll:COREDLL.dll
 0003:0000008c       __imp_Sleep                0010908c     coredll:COREDLL.dll
 0003:00000090       __imp_InsertMenuW          00109090     coredll:COREDLL.dll
 0003:00000094       __imp_wcslen               00109094     coredll:COREDLL.dll
 0003:00000098       __imp__purecall            00109098     coredll:COREDLL.dll
 0003:0000009c       __imp_RaiseException       0010909c     coredll:COREDLL.dll
 0003:000000a0       __imp___C_specific_handler 001090a0     coredll:COREDLL.dll
 0003:000000a4       __imp_DeleteCriticalSection 001090a4     coredll:COREDLL.dll
 0003:000000a8       __imp_free                 001090a8     coredll:COREDLL.dll
 0003:000000ac       __imp_EventModify          001090ac     coredll:COREDLL.dll
 0003:000000b0       __imp_strlen               001090b0     coredll:COREDLL.dll
 0003:000000b4       __imp_??0exception@std@@QAA@PBD@Z 001090b4     coredll:COREDLL.dll
 0003:000000b8       __imp_?what@exception@std@@UBAPBDXZ 001090b8     coredll:COREDLL.dll
 0003:000000bc       __imp_??1exception@std@@UAA@XZ 001090bc     coredll:COREDLL.dll
 0003:000000c0       __imp_CreateEventW         001090c0     coredll:COREDLL.dll
 0003:000000c4       __imp_SendMessageTimeout   001090c4     coredll:COREDLL.dll
 0003:000000c8       __imp_memcpy               001090c8     coredll:COREDLL.dll
 0003:000000cc       __imp___rt_udiv            001090cc     coredll:COREDLL.dll
 0003:000000d0       __imp___CxxThrowException  001090d0     coredll:COREDLL.dll
 0003:000000d4       __imp_??_7type_info@@6B@   001090d4     coredll:COREDLL.dll
 0003:000000d8       __imp_??0exception@std@@QAA@ABV01@@Z 001090d8     coredll:COREDLL.dll
 0003:000000dc       __imp_LocalReAlloc         001090dc     coredll:COREDLL.dll
 0003:000000e0       \177COREDLL_NULL_THUNK_DATA 001090e0     coredll:COREDLL.dll
 0003:000000e4       __imp_PhoneMakeCall        001090e4     phone:PHONE.dll
 0003:000000e8       \177PHONE_NULL_THUNK_DATA  001090e8     phone:PHONE.dll
 0003:000000ec       __imp_tapiRequestMakeCallW 001090ec     Cellcore:cellcore.dll
 0003:000000f0       \177cellcore_NULL_THUNK_DATA 001090f0     Cellcore:cellcore.dll
 0003:000000f4       __imp_RIL_Initialize       001090f4     ril:ril.dll
 0003:000000f8       __imp_RIL_Hangup           001090f8     ril:ril.dll
 0003:000000fc       __imp_RIL_SetEquipmentState 001090fc     ril:ril.dll
 0003:00000100       __imp_RIL_DevSpecific      00109100     ril:ril.dll
 0003:00000104       __imp_RIL_GetRegistrationStatus 00109104     ril:ril.dll
 0003:00000108       __imp_RIL_GetCallList      00109108     ril:ril.dll
 0003:0000010c       __imp_RIL_GetEquipmentState 0010910c     ril:ril.dll
 0003:00000110       __imp_RIL_Deinitialize     00109110     ril:ril.dll
 0003:00000114       \177ril_NULL_THUNK_DATA    00109114     ril:ril.dll
 0003:00000118       __imp_?SWAI_GetRegValue@@YAJPAUHKEY__@@PBG1AAK@Z 00109118     sw_utilityG:sw_utilityG.dll
 0003:0000011c       __imp_?LogV@@YAXPBGZZ      0010911c     sw_utilityG:sw_utilityG.dll
 0003:00000120       __imp_?LogStoreFileLine@@YAXPAGH@Z 00109120     sw_utilityG:sw_utilityG.dll
 0003:00000124       __imp_?GetVerInfo@@YAPAGPAUHINSTANCE__@@@Z 00109124     sw_utilityG:sw_utilityG.dll
 0003:00000128       __imp_?InitLog@@YAXPAUHINSTANCE__@@@Z 00109128     sw_utilityG:sw_utilityG.dll
 0003:0000012c       __imp_?LogC@@YAXPBGZZ      0010912c     sw_utilityG:sw_utilityG.dll
 0003:00000130       __imp_?GetCarrierIndex@@YAKXZ 00109130     sw_utilityG:sw_utilityG.dll
 0003:00000134       \177sw_utilityG_NULL_THUNK_DATA 00109134     sw_utilityG:sw_utilityG.dll
 0003:00000138       __xc_a                     00109138     corelibc:crt0init.obj
 0003:0000014c       __xc_z                     0010914c     corelibc:crt0init.obj
 0003:00000150       __xi_a                     00109150     corelibc:crt0init.obj
 0003:00000154       __xi_z                     00109154     corelibc:crt0init.obj
 0003:00000158       __xp_a                     00109158     corelibc:crt0init.obj
 0003:0000015c       __xp_z                     0010915c     corelibc:crt0init.obj
 0003:00000160       __xt_a                     00109160     corelibc:crt0init.obj
 0003:00000164       __xt_z                     00109164     corelibc:crt0init.obj
 0003:0000016c       ?gSrvState@@3KA            0010916c     DialParsExtOEM.obj
 0003:00000174       ?m_SrvState@CModemStatus@@2KA 00109174     winmodemstat.obj
 0003:00000178       ??_R0?AVbad_alloc@std@@@8  00109178     winmodemstat.obj
 0003:00000194       ??_R0?AVexception@std@@@8  00109194     winmodemstat.obj
 0003:000001b0       ??_R0?AVlength_error@std@@@8 001091b0     winmodemstat.obj
 0003:000001d0       ??_R0?AVlogic_error@std@@@8 001091d0     winmodemstat.obj
 0003:000001f0       __security_cookie_complement 001091f0     corelibc:seccook.obj
 0003:000001f4       __security_cookie          001091f4     corelibc:seccook.obj
 0003:00000200       ??_R0?AVout_of_range@std@@@8 00109200     libcpmt:string.obj
 0003:00000220       _pRawDllMain               00109220     atls:atlbase.obj
 0003:00000228       ?gPwrState@@3W4ePowerState@CModemStatus@@A 00109228     DialParsExtOEM.obj
 0003:0000022c       ?m_nCarrier@@3HA           0010922c     DialParsExtOEM.obj
 0003:00000230       ?g_hmodThisDll@@3PAUHINSTANCE__@@A 00109230     DialParsExtOEM.obj
 0003:00000234       ?bRequestMakeCall@@3HA     00109234     DialParsExtOEM.obj
 0003:00000238       ?bEndCallWorkaround@@3HA   00109238     DialParsExtOEM.obj
 0003:0000023c       ?bRoamMsgCheck@@3HA        0010923c     DialParsExtOEM.obj
 0003:00000240       ?ghwndRilMessage@@3PAUHWND__@@A 00109240     DialParsExtOEM.obj
 0003:00000244       ?g_PowerSaveMode@@3W4RIL_PWRSV_MODES@@A 00109244     DialParsExtOEM.obj
 0003:00000248       ?g_cRefDLL@@3IA            00109248     DialParsExtOEM.obj
 0003:0000024c       ?g_idCmdExternal@@3IA      0010924c     DialParsExtOEM.obj
 0003:00000250       ?gModemstat@@3VCModemStatus@@A 00109250     DialParsExtOEM.obj
 0003:00000254       ?m_bInitFailed@CAtlBaseModule@ATL@@2_NA 00109254     resultelement.obj
 0003:00000258       ?m_MsgBoxBuffer@CModemStatus@@1UtagMsgBoxContent@@A 00109258     winmodemstat.obj
 0003:0000066c       ?m_NonDataCallStatus@CModemStatus@@2KA 0010966c     winmodemstat.obj
 0003:00000670       ?m_DataCallStatus@CModemStatus@@2KA 00109670     winmodemstat.obj
 0003:00000674       ?m_CallType@CModemStatus@@2KA 00109674     winmodemstat.obj
 0003:00000678       ?m_PwrState@CModemStatus@@2W4ePowerState@1@A 00109678     winmodemstat.obj
 0003:0000067c       ?m_RoamState@CModemStatus@@2KA 0010967c     winmodemstat.obj
 0003:00000680       ?m_IsOTASPCommited@CModemStatus@@2HA 00109680     winmodemstat.obj
 0003:00000684       ?m_LastCallEndStatus@CModemStatus@@2GA 00109684     winmodemstat.obj
 0003:00000688       ?m_hApi@CModemStatus@@1PAXA 00109688     winmodemstat.obj
 0003:0000068c       ?m_hActiveWindow@CModemStatus@@2PAUHWND__@@A 0010968c     winmodemstat.obj
 0003:00000690       ?m_MainWndH@CModemStatus@@1PAUHWND__@@A 00109690     winmodemstat.obj
 0003:00000694       ?m_hCurrModPowerState@CModemStatus@@2PAXA 00109694     winmodemstat.obj
 0003:00000698       ?m_hEquipmentStateOn@CModemStatus@@2PAXA 00109698     winmodemstat.obj
 0003:0000069c       ?m_bDMMode@CModemStatus@@1HA 0010969c     winmodemstat.obj
 0003:000006a0       ?m_cFuncResultList@CModemStatus@@1V?$list@VCResultListElement@@V?$allocator@VCResultListElement@@@std@@@std@@A 001096a0     winmodemstat.obj
 0003:000006ac       ?_pAtlRawDllMain@@3P6AHPAXK0@ZA 001096ac     atls:atlbase.obj
 0003:000006b0       ?_AtlModuleInstance@ATL@@3PAUHINSTANCE__@@A 001096b0     atls:atlbase.obj
 0003:000006b4       ?_AtlBaseModule@ATL@@3VCAtlBaseModule@1@A 001096b4     atls:atlbase.obj
 0003:000006e8       __onexitend                001096e8     <common>
 0003:000006ec       __onexitbegin              001096ec     <common>
 0003:000006f0       _exitflag                  001096f0     <common>

 entry point at        0001:0000399c

 Static symbols

 0001:00000090       __unwind$39846             00101090 f   clsfact.obj
 0001:000020a0       __catch$61851              001030a0 f i winmodemstat.obj
 0001:000020cc       __catch$61849              001030cc f i winmodemstat.obj
 0001:0000283c       __unwind$62693             0010383c f   winmodemstat.obj
 0001:000028c0       __unwind$63006             001038c0 f i winmodemstat.obj
 0001:00002a10       __unwind$63144             00103a10 f i winmodemstat.obj
 0001:00002a94       __unwind$63233             00103a94 f i winmodemstat.obj
 0001:00002c10       __unwind$63394             00103c10 f   winmodemstat.obj
 0001:00002c28       __unwind$63395             00103c28 f   winmodemstat.obj
 0001:00002cf0       __catch$63550              00103cf0 f   winmodemstat.obj
 0001:00002e24       __catch$63589              00103e24 f   winmodemstat.obj
 0001:000033d0       __catch$63853              001043d0 f   winmodemstat.obj
 0001:000034fc       __catch$63895              001044fc f   winmodemstat.obj
 0001:00003bc4       doexit                     00104bc4 f   corelibc:crt0dat.obj
 0001:00003f24       ?CanThisExceptionObjectBeDestructed@@YAEPAUEHExceptionRecord@@E@Z 00104f24 f   LIBCMT:frame_ce.obj
 0001:00004270       ?CallCatchBlock@@YAPAXPAUEHExceptionRecord@@PAKPAU_CONTEXT@@PBU_s_FuncInfo@@PAXHK@Z 00105270 f   LIBCMT:frame_ce.obj
 0001:00004608       ?BuildCatchObject@@YAXPAUEHExceptionRecord@@PAKPBU_s_HandlerType@@PBU_s_CatchableType@@@Z 00105608 f   LIBCMT:frame_ce.obj
 0001:000047dc       ?FindHandler@@YAEPAUEHExceptionRecord@@PAKPAU_CONTEXT@@PAU_DISPATCHER_CONTEXT@@PBU_s_FuncInfo@@H@Z 001057dc f   LIBCMT:frame_ce.obj
 0001:000053d4       __unwind$17778             001063d4 f   libcpmt:string.obj
 0001:00005464       __unwind$17968             00106464 f   libcpmt:string.obj
 0001:00005794       ??__EgModemstat@@YAXXZ     00106794 f   DialParsExtOEM.obj
 0001:000057b4       ??__E?m_cFuncResultList@CModemStatus@@1V?$list@VCResultListElement@@V?$allocator@VCResultListElement@@@std@@@std@@A@@YAXXZ 001067b4 f   winmodemstat.obj
 0001:000057e8       ??__E_AtlBaseModule@ATL@@YAXXZ 001067e8 f   atls:atlbase.obj
 0001:00005824       ??__FgModemstat@@YAXXZ     00106824 f   DialParsExtOEM.obj
 0001:00005830       ??__F?m_cFuncResultList@CModemStatus@@1V?$list@VCResultListElement@@V?$allocator@VCResultListElement@@@std@@@std@@A@@YAXXZ 00106830 f   winmodemstat.obj
 0001:00005858       ??__F_AtlBaseModule@ATL@@YAXXZ 00106858 f   atls:atlbase.obj
